:100000000EC028C027C026C025C024C023C022C0DF
:1000100021C020C01FC01EC01DC01CC01BC0112499
:100020001FBECFE5D1E0DEBFCDBF10E0A0E6B0E05F
:10003000E0EBF0E002C005900D92A036B107D9F7D1
:1000400010E0A0E6B0E001C01D92A036B107E1F7D4
:100050000FD02CC0D5CF382F882349F020E040E2C4
:100060005EE4CA010197F1F72F5F2317D0F30895DB
:10007000CF93DF9388E187BB18BAC8E3D0E08881CB
:1000800083FF04C08881877F888303C0888188605C
:100090008883888184FF04C088818F7E888303C021
:1000A00088818061888384E6D6DFE9CFF894FFCF2A
:00000001FF
